:100000008A01203084004C29D92870088207FC29F5
:10001000FC293B2D0E281F283028352EC71F822291
:10002000471FFC2947137108053C031CFC29710874
:100030008207FC29AC2DB62DB82DC22DC42DC71FAB
:100040008222471FFC2947137108053C031CFC2929
:1000500071088207FC29FC29FC29D42DDE2DE02D16
:10006000C71F8222471FFC29471371080E3C031C3F
:10007000FC2971088207FC29FC29FC29F32DFD2DA0
:10008000FF2D012E032E082E182EFC291A2E242EA9
:10009000262E302E74088207412C472C5F2C682CAA
:1000A000712C972C972C972C972C972C972C972C5E
:1000B000972C972C74088207412CA42CA42CA42CD8
:1000C000D72CD72CD72CD72CD72CD72CD72CD72C18
:1000D000D72CD72C1A08FC001819D3289818D32825
:1000E000C71BD528471AD5287408031DD5287C08B6
:1000F0000B237008820782288A288F288F288F2850
:100100008F288F286708031D98287C08243C031932
:10011000B42898286708063C0319B92898287C0851
:100120002C3C0319BD287C082A3C0319BD289828BB
:100130007C08083C031DA528E7080319B328E7033A
:1001400020300B2308300B23B3286708A03E84001F
:100150007C08800087110A3C0319C72867081F3CE8
:10016000031CC728E70A08000130F000F101E7018D
:10017000A5280230F000E7010800F10A6708A03E58
:1001800084007C088000E701471787110800871565
:10019000E701F1014713F008031DD1280630F000F4
:1001A0000800F0010800181218164713E701F001C3
:1001B0000800FE00030E8301FF000408FD000B1180
:1001C00084308100ED2030218C1A6A207D08840063
:1001D0007F0E8300FE0E7E0E0900A30DA009A1096B
:1001E00020081507A00021080318210A1607A100FE
:1001F000A11DFD280310A10CA00C06302102F13036
:10020000031920020318072905292310082923149C
:100210001508A0001608A100A40B22290A30A4008A
:10022000C9010830CA00A30D0318C90ACA0B132953
:10023000A30DA50D053049020318202925142129F5
:100240002510A60A0F302302031D080005302402E2
:1002500003192F29031C2E29A4030800A40A08004F
:10026000AF03031D3929C60A6E084602031D39294A
:10027000C601B10D07183E2931103F293114A20DD6
:10028000071A4429221045292214BE0D051A4A29AD
:100290003E104B293E1408008001840A841F4C291B
:1002A0003E14311422140230EE0003178F010313A1
:1002B0000A30A4001E308500860187018316D330E2
:1002C000810006309F00850105168601B530870044
:1002D00083120730970010148316033092008312A4
:1002E0000F309D0001309B001215831619309900C4
:1002F00098168312181398171816312260308B0045
:1003000097302622AE01A701A801A9014712C71004
:10031000F621783C031D8229F408031D8229471623
:10032000EA21333C031D8229EA21783C031D8229FE
:10033000B5018E227622C713963026222908AA00FC
:100340002808A9008711EA21A8008715EA21A7003B
:10035000783C03199E292E08A13E26224719A7178B
:100360002708F526D200A7134719AA172A08F52649
:10037000AC00AA13D2080319CA29AC080319D12961
:1003800052082C020319C529DD29AE080319D12909
:10039000AE03D1292A08A7002C08D200D2080319DD
:1003A000DD2952084C3C031DD7294711E129520889
:1003B000463C031DE0294715E129AE0A5F30D20013
:1003C00011232A08783C031980292E08063C031DB6
:1003D0009E2980298B1700008B132608063C0318E2
:1003E000EA29A60125087F398B1708008B17871A81
:1003F000FB292324E82405288B13A6080319F629D2
:10040000A60125087F398B170800871A0800831674
:10041000FF308600831285168515851005110608A4
:1004200005150339033C031D0D2A85148511831618
:10043000860183120800871A0800B80005223808D0
:10044000860085118512051105150800871A080018
:10045000B800052238088600851585120511051596
:1004600008003D304926363049260514A122642271
:1004700076228E2264228E2228301B2200301B22FC
:100480004130262280302622A130262200301B2235
:100490001B2221302622523088256530882576306F
:1004A000882520308825313088252E308825343025
:1004B00088258E2208002830B20000301B22C03070
:1004C0002622B20B5D2A08004030B2000230B30091
:1004D00000301B22C0302622B20B682AB30B682AD8
:1004E00008002830C107031C762AC20A4108C3004D
:1004F0001B224208C4001B22403026223608370245
:10050000C5000800A0301B221E301B2240302622CE
:1005100008002830BF07031C8E2AC00A3F081B2290
:1005200040081B222430262208002830E807031C3C
:100530009A2AE90A68081B2269081B22243026220D
:100540000800A030E8001E30E9009A2AAB00360807
:100550003702C5002B08443C0319CE2AC71CB72A12
:10056000C7102B08203C0319B72AF123BE2AB5086F
:10057000031DBE2A2B08203C0319DF2AB50A2030B0
:100580002B021B22C03026223508273C0318DF2A05
:10059000C714B501B60AB70A8922D62AB5080319C5
:1005A000DF2AC710B501B60AB70A89223708C33C4B
:1005B000031CEE2A3608073C031CE72AE02AC71072
:1005C00035081B2236081B2221302622080007305E
:1005D000B600C50A71225B228E22E02AB601B5015F
:1005E000C101C201C301C401BF01C001B701C501FE
:1005F00076228E2264228E224714DF2A53080A3C78
:10060000031D042B2030D30053080D3C031D0A2B7F
:100610002030D30008008316981C0C2B83129900FD
:1006200008005208413C0319F02B5208423C0319C0
:10063000F02B1430B200653084000008840A80007A
:1006400084038403B20B1D2B5B087A3C031DCB2B68
:100650005A08633C031DCB2B59087A3C031DCB2B56
:100660005808633C031DCB2B5708203C031DCB2BA4
:100670002630F300E9262A3C03194E2B7208560255
:1006800003194E2B2730F300E926560203194E2B8F
:100690002830F300E9265602031DCA2B65305502A7
:1006A0000319B62B623055020319B62B643055027C
:1006B0000319B62B2930F300E926793C031D642B7E
:1006C000613055020319B62B2A30F300E926793C34
:1006D000031D6E2B633055020319B62BF30AE9266E
:1006E000793C031D772B663055020319B62BF30AAC
:1006F000E926793C031D802B673055020319B62B80
:10070000F30AE926793C031D892B68305502031949
:10071000B62BF30AE926793C031D922B693055026A
:100720000319B62BF30AE926793C031D9B2B6A308B
:1007300055020319B62BF30AE926793C031DA42BB5
:100740006B3055020319B62BF30AE926793C031DD9
:10075000AD2B6C3055020319B62BF30AE926793C10
:10076000031DCA2B7A305502031DCA2BC719CB2B88
:10077000C7154430A6220930B2005B30840000085F
:100780000B23FE220008A6228403B20BBF2B4430A9
:10079000A6220800C71156086E3C031DE92B550818
:1007A0006E3C031DE92B54086E3C031DE92B5308D6
:1007B0006E3C031DE92BC71D080053080B230D30A9
:1007C0000B230A300B235308A6224430A622C7115C
:1007D0000800C71DF02B53080B23FE225308A62246
:1007E00008005408203C03190800B50A1230B20072
:1007F000553084000008203C0319042CB50A840AF3
:10080000B20BFA2BB50108003508B200B20A00306D
:100810001B22C2302622B20B072C8E225330350702
:1008200084003508B200203000021B22C03026228E
:100830008403B20B132C08006C081B226D081B22CA
:10084000213026220800BE08031D392CC608031DCE
:10085000412CC60AF40A87110430EE0074080E3CDD
:100860000319332C4A28A1226422F4017622E022C3
:10087000C7133E08310522050319412CE708031967
:100880008715080053308825543088250800973094
:100890002622A13026220430EC00ED011C24263053
:1008A000EB00A12264229A22822242243130882540
:1008B0003A3088256B08F300E9269F24412CED0A85
:1008C0001C242730EB009522422432308825582CF6
:1008D000ED0A1C242830EB00952242243330882571
:1008E000582CEC01ED0AED0A1C2495224130882594
:1008F000433088254630882547308825483088256C
:10090000493088254A3088254B3088254C30882549
:100910005A30882595222930EB00F3000A30B200C6
:10092000E9268825F30AB20B902C9A22412CEC0A76
:100930001C246B08F300E9268825EB0A412CE03ED5
:100940001B22C43026220800A2080319C32CB108B8
:100950000319AB2C08006B08E926EA002A3C0319AE
:10096000B82C6A08793C0318BA2C2A30EA00BB2C50
:100970006030EA00EA0A6A08F2006B08F300D22647
:100980006A089F2408006B08E926EA002A3C03193C
:10099000D02C6A08613C031CD22C2A30EA00D32CEC
:1009A0007B30EA00EA036A08F2006B08BE2C6B0891
:1009B000F300E926793C031DDF2C6E30E02C793002
:1009C000EA00F2006B08F300D2266A089F240800B0
:1009D000C608031D3A2DC60AB1080319F32CA20854
:1009E0000319172D392C8711F408031D5A28C7172E
:1009F00034250230EE0094302622370845020319D0
:100A00003A2DC50803190A2DC5032830C302031C5B
:100A1000C403342D471C3A2DBC30370203183A2D3D
:100A2000BC30C5006030C3001D30C400342D8711B8
:100A3000F408031D5A2834250230EE009430262293
:100A4000360837024502031D272DC7130800BB30A7
:100A500045020318312DC50A2830C3070318C40AFC
:100A6000342DC501C301C40143081B2244081B22C5
:100A700040302622080094302622A330840000084B
:100A8000473C031D562D840A00084C3C031D562D7F
:100A9000840A00084C3C031D562D0330F000A030A2
:100AA0001B221E301B2224302622FC29A330840066
:100AB0000008563C031D6F2D840A0008543C031D9A
:100AC0006F2D840A0008473C031D6F2D0430F00091
:100AD000F0301B221E301B2224302622FC29A3309A
:100AE00084000008413C031DFC29840A0008503C96
:100AF000031DFC29840A0008423C031DFC29053023
:100B0000F00040301B221F301B2224302622FC29FB
:100B1000B400E03E1B22C030262234080800A0307A
:100B2000840000082C3C03199D2D00082A3C031961
:100B30009D2D00088825840A912D203088250800E5
:100B4000A030840000082E3C0319AA2D0008882537
:100B5000840AA22D840A08004C308825413088255B
:100B6000543088253A3088258F25FC298F25FC298B
:100B70004C3088254F3088254E3088253A308825DE
:100B80008F25FC298F25FC29B8301B221F301B2202
:100B90002430262255308825543088254330882536
:100BA0003A308825A025FC295430882552308825E4
:100BB0004B3088253A3088258F25FC298F25FC2944
:100BC0005330882550308825443088253A30882590
:100BD0008F254B308825743088252030882588253E
:100BE00088258825FC2958308825543088254530AB
:100BF00088253A3088258F25FC298F25FC298F25CB
:100C0000FC298F25FC298F25882588258825FC2906
:100C100068301B221F301B222430262242308825B8
:100C20004F308825443088253A3088258F25FC2987
:100C30008F25FC294230882550308825443088256E
:100C40003A3088258F25FC298F25FC2948308825B6
:100C500044308825533088253A3088258F25FC2953
:100C60008F25882588258825FC29F001A03084005F
:100C70000008683C0319522E0008703C0319552ED9
:100C80000008733C0319762E00086D3C0319962E5C
:100C9000FC29F300E9260319512E72080B23F30AED
:100CA0004A2E080000304926FC2931300B2332300F
:100CB0000B2333300B2361300B2363300B2366305F
:100CC0000B2367300B2368300B2369300B236A300A
:100CD0000B236B300B236C300B237A300B230D303E
:100CE0000B230A300B2326304926FC29840A0008EE
:100CF000743C031DFC29840A0008313C03198E2E24
:100D00000008323C03198B2E0008333C031DFC29DC
:100D10002830F300902E2730F300902E2630F30079
:100D2000840A840A0008F200D226FC2904308407D1
:100D30002930F3000008613C0319CC2EF30A0008A7
:100D4000633C0319CC2EF30A0008663C0319CC2E31
:100D5000F30A0008673C0319CC2EF30A0008683C2C
:100D60000319CC2EF30A0008693C0319CC2EF30AB0
:100D700000086A3C0319CC2EF30A00086B3C0319E7
:100D8000CC2EF30A00086C3C0319CC2EF30A0008A1
:100D90007A3C0319CC2EFC29840A840A0008F2004C
:100DA000D226FC29031783168C18D42E83127308BD
:100DB0008D0072088C0083168C130C158B13553024
:100DC0008D00AA308D008C140C118B178312031325
:100DD00008000317831273088D0083168C130C14FC
:100DE00083120C080313F20008000A158A140A146F
:060DF000FF268A01080045
:020DFE0082076A
:100E00000034003400340034003400340034003442
:100E100000340034003400340034003400340D3425
:100E200000340034003400340034003400347434AE
:100E30000034003400340A34003420347634003472
:100E400000340034003400340034003400346234A0
:100E50000034003400345F3400344C3478340034CF
:100E600000340034003442340034653446340034F5
:100E700000347534713400346B3400340034003481
:100E800000340034003400340034003400346F3453
:100E9000003400340034683400346E346D3400346F
:100EA0000034003400346C3400347234673400345D
:100EB0000034693470340034633400340034003456
:100EC0000034003400347A340034643400340034A4
:100ED0000034733479340034663400340034003420
:100EE00000346134773400346A3400340034003420
:100EF0004134003400340034003400340034003411
:100F00000034003400340034003400340034003441
:100F100000340034003400340034003400340D3424
:100F200000340034003400340034003400343534EC
:100F30000034003400340A34003420343D340034AA
:100F400000340034003400340034003400343F34C2
:100F50000034003400345F3400344C342F34003417
:100F60000034003400344234003433344634003426
:100F70000034373431340034283400340034003441
:100F80000034003400340034003400340034393488
:100F9000003400340034233400342C342E34003434
:100FA000003400340034293400343434263400341E
:100FB00000343834303400343A34003400340034EF
:100FC0000034003400342B34003424340034003432
:100FD00000345C34363400343F34003400340034A0
:100FE00000342D3432340034003400340034003402
:100FF0004134003400340034003400340034003410
:02400E00723FFF
:10420000730074006E003D005B0061002C002A000A
:104210005D000D000A006D00730067005F0078000C
:104220003D005B0079002C006E005D000D000A006F
:104230007000720069006E0074000D000A006800D2
:1042400065006C0070000D000A0000002A00680084
:104250006A00790079006E006E006E006E006E00DC
:104260006E006E006E000D000A0000005200650036
:104270007600200031002E0034000D000A000000FE
:00000001FF
